:100000008A110A1205280000090083160E309F008D
:10001000810164308F00831241309F0083160130CC
:1000200085000F30860083123014B014BD01BE016C
:1000300006158615B901BA01BB01BC01B101B201B7
:10004000B301B4010A30A000A1019D220511851160
:100050008316051185110F30860583120230A0002A
:100060000030A1009D2233300A2333300A2333307D
:100070000A2322300A2328300A230F300A230130B2
:100080000A2301300A237430F3226530F3226D30E5
:10009000F3227030F3227330F3222830F3225330EE
:1000A000F3222930F3223F30F3222030F3220619C5
:1000B0003014061D30108619B014861DB01030188B
:1000C00085283D08013EBD003E080318013E003E64
:1000D000BE00051601300A233D08A4003E08A50015
:1000E0001F232030F3225330F3229030A000013040
:1000F000A1009D2205129030A0000130A1009D2298
:1001000006193014061D30105F281F308305B01803
:10011000AD283D080A3EBD003E080318013E003EE2
:10012000BE00051601300A233D08A4003E08A500C4
:100130001F232030F3225330F3229030A0000130EF
:10014000A1009D2205129030A0000130A1009D2247
:100150008619B014861DB01087281F308305061835
:100160005F29E3211430A000A1019D223708A000DF
:100170003808A100FF30A200A3015F22B9002108C6
:10018000BA003708A0003808A100FF30A200A30180
:100190005F222408BB002508BC003908B500F22105
:1001A0004608CD004408CC000530AE008030AF00DA
:1001B0008316851383120530AC004030AD008316E2
:1001C000051383125A235A235723A0303E233208A3
:1001D0003E2331083E234C083E235A231430A0000E
:1001E000A1019D223108013EB10032080318013EF1
:1001F000003EB2003B08B5000530AE008030AF00D5
:100200008316851383120530AC004030AD00831691
:10021000051383125A235A235723A0303E23320852
:100220003E2331083E234D083E235A231430A000BC
:10023000A1019D2201300A232830F3224530F32208
:100240002E30F3223108A4003208A5001F232930E4
:10025000F3222030F3223D30F3222030F3224C08E9
:10026000A400A5011F232C30F3224D08A400A501F2
:100270001F233108013EB10032080318013E003E41
:10028000B2000130C000C1014008A0004108A10037
:100290003E08A3003D088A22031D5D29E830A00026
:1002A0000330A1009D220130C00700300318013E39
:1002B00003185D29C107031C44291F3083051F3023
:1002C00083058618DF291430A000A1019D22053086
:1002D000AE008030AF008316851383120530AC006A
:1002E0004030AD008316051383125A235A23572337
:1002F000A0303E2334083E2333083E235A2357239D
:10030000A1303E238423CC005A231430A000A10145
:100310009D223308013EB30034080318013E003E1D
:10032000B4000530AE008030AF0083168513831211
:100330000530AC004030AD008316051383125A23FC
:100340005A235723A0303E2334083E2333083E234C
:100350005A235723A1303E238423CD005A2314303F
:10036000A000A1019D2201300A232830F3224C3045
:10037000F3222E30F3223308A4003408A5001F23F3
:100380002930F3222030F3223D30F3222030F322B3
:100390004C08A400A5011F232C30F3224D08A40013
:1003A000A5011F233308013EB30034080318013EA2
:1003B000003EB400D030A0000730A1009D221F30C5
:1003C00083055728E2291F1483169F171F13003037
:1003D0008312A000E22283161E088312B7001E08B3
:1003E000B80008003908A6003A08A700FF30A200AC
:1003F000A3014922B7002508B80037083B07B7001A
:1004000038080318013E3C07B8003708A600380832
:10041000A7001430A200A3014922C4002508C5008A
:100420004408A0004508A1009830A2000130A300B4
:100430005F22C4002108C5003708A6003808A700BD
:100440001430A200A3014922C6002508C7004608AF
:10045000A0004708A1009830A2000130A3005F224D
:100460002408C6002508C7003708A0003808A100E6
:10047000A30114308422031D412AC401C501C60111
:10048000C7011F3083050A30A000A1019D2208008A
:10049000482A1030A800A101A001A70CA60C031C3B
:1004A000572A2208A00723080318230FA107A10C2D
:1004B000A00CA50CA40CA80B4D2A24080800103091
:1004C000A600A501A401210DA40DA50D2208A402DA
:1004D0002308031C230FA5020318752A2208A4076A
:1004E00023080318230FA5070310A00DA10DA60BC9
:1004F000632A20080800A20005308D2AA2000230DD
:100500008D2AA20006308D2AA20003308D2AA20077
:1005100004308D2AA20001308D2AA8002308210270
:10052000031D942A22082002043003180130031905
:1005300002302805031DFF300800A0080319A82A6F
:10054000AF22A003000000000000000000009D2A70
:10055000A10803190800AF22A103A0039D2A0C30B3
:10056000A500A50BB12A000000001230A200A20BCA
:10057000BE2AC022C022000000000800C022B72A04
:100580000D30A400A40BC22A000008000A30A80203
:10059000031C0800CB2A0630A802031C0800CB2A43
:1005A0001030A8020001031C013EA902031C080030
:1005B000D92A0A30A8020001031C013EA902031C2B
:1005C0000800D92AA00DA00DA00D3830A005C1301B
:1005D00020049F001430A800C6221F151F19EE2A00
:1005E0000C131F100800A80085150F308605280879
:1005F000F03986040623A80E0F3086052808F03946
:10060000860406233230A800C62208000515000023
:1006100005110800A80085110F3086052808F0395B
:1006200086040623A80E0F3086052808F0398604B4
:100630000623D030A8000730A900D0220800A71751
:100640002730A300103030230330A300E8303023DC
:10065000A30164303023A3010A30302324083B2B4C
:10066000A2002508A1002408A0005F222008031D85
:10067000A713A71B0800303EF3220800A000083093
:10068000A100A00D03185D23031C622367236C23C4
:10069000A10B412B78234F237E236223080067237D
:1006A0002E0884002F080005FF3E6C2308006223FB
:1006B0006C23752B67235D23752B2E0884002F0870
:1006C0008004712B2E0884002F098005712B2C08C3
:1006D00084002D088004712B2C0884002D098005CE
:1006E000712B8417000984138005000000000800A6
:1006F0002E08840084172F08800408002E08840028
:1007000084172F098005080078230830A1004F23A3
:10071000A00DA10B872B7E235D2367236C2362230F
:100720002008080078230830A1004F23A00DA10B5A
:0E073000952B7E23622367236C23200808008C
:02400E00702F11
:00000001FF
